:020000040002F8
:10800000B8500020D9830200E1830200E38302001C
:10801000E5830200E7830200E9830200000000001C
:10802000000000000000000000000000C583020006
:10803000ED83020000000000EF830200F1830200E4
:10804000F3830200F3830200F3830200F383020050
:10805000F383020000000000F3830200F3830200B8
:10806000F3830200F3830200F3830200F383020030
:10807000F3830200F3830200F3830200F383020020
:10808000AD96020049940200F3830200F3830200DC
:10809000F3830200F3830200BD940200F383020025
:1080A000F3830200F38302000000000000000000E0
:1080B000F3830200F38302000000000000000000D0
:1080C00000000000000000000000000000000000B0
:1080D00000000000000000000000000000000000A0
:1080E0000000000000000000000000000000000090
:1080F0000000000000000000000000000000000080
:10810000000000000000000000000000000000006F
:10811000000000000000000000000000000000005F
:10812000000000000000000000000000000000004F
:10813000000000000000000000000000000000003F
:10814000000000000000000000000000000000002F
:10815000000000000000000000000000000000001F
:10816000000000000000000000000000000000000F
:1081700000000000000000000000000000000000FF
:1081800000000000000000000000000000000000EF
:1081900000000000000000000000000000000000DF
:1081A00000000000000000000000000000000000CF
:1081B00000000000000000000000000000000000BF
:1081C00000000000000000000000000000000000AF
:1081D000000000000000000000000000000000009F
:1081E000000000000000000000000000000000008F
:1081F000000000000000000000000000000000007F
:10820000DFF810D000F03AF900480047B9A60200A4
:10821000AFF30080B850002030B450E8012F93B283
:10822000C48923448489A34228BF1B1B0489A34219
:1082300002BFBFF32F8F002007E0C3EA020340E82C
:108240000134002CE9D14FF001000A6030BC7047C6
:1082500050E8012FC2EA024240E801210029F7D18B
:10826000704730B450E8022F1FFAA2F3C488A3422B
:1082700002BFBFF32F8F00200DE0C48923448489FF
:10828000A34228BF1B1BC2EA034340E80234002C70
:10829000E8D14FF001000A6030BC704750E8022F6F
:1082A000C2EA224240E802210029F7D17047034682
:1082B00053E8022FD988B2EB324F4FF0000017BFBE
:1082C00092B241EA014142EA014104E05A68B2EB4C
:1082D000324F08BF012043E80212002AE8D170475C
:1082E00030B4044654E8000F0D4644E80053002B18
:1082F000F8D1156030BC704730B4044654E8000F24
:1083000040EA010544E80053002BF7D1156030BC6A
:10831000704730B4044654E8000F00EA010544E811
:108320000053002BF7D1156030BC704730B40446C1
:1083300054E8000F80EA010544E80053002BF7D110
:10834000156030BC704730B4044654E8000F00EBB1
:10835000010544E80053002BF7D1156030BC70478D
:1083600030B4044654E8000FA0EB010544E8005384
:10837000002BF7D1156030BC704770B404464FF045
:10838000000054E8006F0D68AE4207BF44E80023C8
:10839000012044E800630E60002B1CBF0020F0E7C2
:1083A00070BC704730B4044654E8000F88422CBFBC
:1083B000451A054644E80053002BF5D1156030BC42
:1083C000704700001EF0040F0CBFEFF30880EFF3BE
:1083D000098003F07DBC000006488047064800473E
:1083E000FEE7FEE7FEE7FEE7FEE7FEE7FEE7FEE765
:1083F000FEE7FEE7C194020001820200202A04DBAE
:10840000203A00FA02F1002070479140C2F12003A7
:1084100020FA03F319439040704740EA01039B0799
:1084200003D009E008C9121F08C0042AFAD203E0E9
:1084300011F8013B00F8013B521EF9D27047D2B24D
:1084400001E000F8012B491EFBD270470022F6E73D
:1084500010B513460A4604461946FFF7F0FF2046BA
:1084600010BD30B504460020034600E05B1C93427B
:1084700003D2E05CCD5C401BF8D030BD064C074D0C
:1084800006E0E06840F0010394E8070098471034E4
:10849000AC42F6D3FFF7B8FECCDA0200ECDA020009
:1084A0002DE9F04F8BB0DDE914B94D46144615F9AE
:1084B000046B00961F4680468A462B46024621469C
:1084C00002A800F08EFC02A94A46084600F085FC8E
:1084D0004B4602AA4146404600F06FFC4B4602AABA
:1084E0002146204600F069FC2B4652463946384664
:1084F000009600F076FC4A46394602A800F06DFC72
:1085000002A92B4642460846009600F06AFC02A9E2
:108510002B4622460846009600F063FC2B46424656
:1085200021462046009600F05CFC4B462246514610
:10853000504600F042FC2B4602AA4146584600969F
:1085400000F04FFC4B465A463946384600F035FCA1
:108550002B46524639463846009600F042FC3246D9
:1085600002A9204600F004FE0BB0BDE8F08FF0B584
:10857000154689B01C4607460E461A4629466846E7
:1085800000F02BFC23466A463946384600F015FCBD
:1085900023462A466946684600F00FFC23466A4691
:1085A0003146304600F009FC09B0F0BD8B1802449A
:1085B0008B4200D1704713F8010D02F8010DF7E767
:1085C0002DE9F0479846B3F90230894613F11F01AF
:1085D00048BF03F13E01DD1D48BF03F10E05EC105D
:1085E0004E11944275B228BF14462946074600F042
:1085F0007BFA22464946FFF7D9FFB8F90230B3EBC0
:10860000C40F4FEAC40220D2D21A07EB8601002021
:10861000C2F120068F420FD308F124082A463946BA
:10862000404600F06CFA01280FD02B4642463846EF
:10863000BDE8F04700F0ACBD51F8044D24FA02F358
:1086400003430B6004FA06F0E4E7BDE8F0872DE988
:10865000F04793F9006092B00446894610463146CF
:1086600015461F4600F060FA002840F091803A4617
:10867000494602A800F0B1FB3B4602AA21460AA8DF
:1086800000F09BFB02A908463A4600F0A6FB3B46D9
:108690002A464946484600F090FB07F104083A464E
:1086A0002946284600F099FB43462A4621462046A3
:1086B000009600F048FA43462A4629462846009686
:1086C00000F041FA43462A4621462846009600F02B
:1086D00088FB3B462A462146204600F06EFB434677
:1086E000224621462846009600F02DFA4346009681
:1086F0002A462146204600F026FA2368DB074AD5A1
:10870000334642462146204600F0C2F931468246B1
:10871000204600F020FD06F18043013B54F8232061
:1087200042EACA7244F823203A462146284600F01D
:1087300054FB43460AAA29462846009600F051FBFE
:1087400043460AAA29462846009600F04AFB0AA991
:10875000084643462A46009600F043FB3B460AAAD9
:108760002146204600F029FB02AA43461046214636
:10877000009600F036FB32462946204600F0F8FC11
:108780004946284600F0F4FC02A9484600F0F0FCF7
:1087900012B0BDE8F0873146204600F0DCFCC3E7AC
:1087A000004870471CDA02002DE9F04FEFB00025B9
:1087B000789E04911946B6F90230069013F11F070E
:1087C00048BF03F13E0747F3471707F1FF3926ABD0
:1087D0004EA843F829506EAB03EB8903924696F9F5
:1087E000012043F8805C43F8605C96F90040FFF795
:1087F000DDFE96F9012056A81144FFF7D7FE214669
:108800004EA800F091F98046002840F03A8156A821
:1088100000F08AF90390002840F0358106F1240B1E
:108820003A464EA9584600F06AF9012840F02D81D9
:108830003A4656A9584600F062F90128089040F0DF
:1088400024811EAD0DF138083B465A4656A92846EC
:1088500000F092F9039B48F82930524640460499AB
:108860003346FFF7ADFE414640465B462A46009739
:1088700000F005FA0DF5BC795B462A464EA916A80C
:10888000009700F0FCF922464846069900F070FC7B
:10889000A300099309EB84030493069B049803EB5C
:1088A000840100F065FC0DF1D80A06F14403194675
:1088B0005046059300F05CFC059BA10059183EA8AA
:1088C00000F056FC331D5246494628460094079353
:1088D00000F087FA4A465046CDE900A6049B3EA91F
:1088E000FFF7DEFD2346321D2946284600F044F9F5
:1088F0003346484604992A46FFF739FE039A0A92FE
:10890000059A0B92069A39464046CDE90C2900F0AB
:1089100003FC3946824616A800F0FEFB8245B8BF2C
:1089200082461FFA8AFA0AF1FF390FFA89F9494695
:10893000404600F05DFC4946B0F1000816A818BF9B
:108940004FF0010800F054FC002814BF0220002062
:1089500048EA00080AAB224653F8281026A800F07F
:1089600007FC0DF1B809A3001944484600F000FCCB
:108970002146284600F0B8F8089B2B6026ABCDE9CD
:108980000435AAF102080FFA88F8B8F1000F24DACA
:108990000599079A0846234600F0EEF8059A0498D0
:1089A00033464946FFF7E3FD04993A46584600F03E
:1089B000A6F8012805D004993B465A46084600F01F
:1089C000E7FB013C64B24EAA23064FD5039BB3FAE2
:1089D00083F040096FB0BDE8F08F3346059A0498E4
:1089E000D6F8A4504946A84741460EA800F000FC1E
:1089F0004146B0F1000A16A818BF4FF0010A00F076
:108A0000F7FB002814BF022000204AEA000A0AAB44
:108A100053F82A1029B30DF1D80A2246504600F027
:108A2000A7FB099B3EA8194400F0A2FB059A334618
:108A30003EA95046FFF79BFD079B049900945246C0
:108A400046A800F0CEF9049A4B463EA95046CDE91F
:108A500000A6FFF725FD0599334646AA084600F013
:108A6000ACF908F1FF380FFA88F88EE7049B52F84A
:108A7000241053F824304B40039919430391013CCF
:108A8000A2E72846A6E74046A4E70398A2E700002D
:108A9000C3F10803DB0070B501330446002003A5D1
:108AA0005B1920C940CAAD1920C4184720C940CA63
:108AB000754120C420C940CA754120C420C940CA9C
:108AC000754120C420C940CA754120C420C940CA8C
:108AD000754120C420C940CA754120C420C940CA7C
:108AE000754120C4404170BD002310B51C465AB2E8
:108AF000914200DC10BD40F823400133F7E710B588
:108B0000013A52B2130601D5002010BD50F82240A0
:108B100051F822309C4205D802F1FF32F2D24FF0D8
:108B2000FF30F2E70120F0E710B500231A465CB2EF
:108B3000A14203DCB2FA82F0400910BD50F8234094
:108B400001332243F3E770B59DF910601D463346AB
:108B50000446FFF79DFF30B9324621462846FFF70D
:108B6000CEFF012807D033462A4621462046BDE8DD
:108B7000704000F00DBB70BDF0B50F46A1B00646C9
:108B80001946384615461C46FFF7CEFF20B1304641
:108B9000FFF7AAFF21B0F0BD22463946684600F033
:108BA000E7FA294608A800F0E3FA10A82146FFF7E3
:108BB0009BFF012318A81093FFF796FF224608A9F0
:108BC0006846FFF79CFF28B9224610A9304600F0FE
:108BD000CFFADFE7009BDA0709D42146684600F0A8
:108BE000BAFA2246294610A800F0E2FBE6E7089B05
:108BF000DB0707D4214608A800F0ADFA2246294633
:108C000018A8F1E7002823461CDD08AA6946684633
:108C100000F0BEFA2146684600F09DFA224618A9E7
:108C200010A8FFF76CFF002805DA10A923462A4692
:108C30000846FFF72DFF10A9234618AA084600F0A2
:108C4000A7FACEE708A96A46084600F0A1FA21462D
:108C500008A800F080FA224610A918A8FFF74FFFD5
:108C6000002805DA18A923462A460846FFF710FF10
:108C700018A9234610AA084600F08AFABEE72DE993
:108C8000F04FB5B004AC9DF9F8501E4680462B4617
:108C9000204600F0B8F824AB29463046CDE902342E
:108CA00000F03AFAC0EB851424B2002C2146B8BF7C
:108CB00004F11F01634241F3471103F01F0314A89D
:108CC00004F01F0758BF5F42FFF70EFF002F08B2E6
:108CD0002BDD14AB002203EB8001C7F1200E1346FD
:108CE000AB4217D36B00019314AB03EB85096F1EE6
:108CF00034AB012603EB8707002C54DA34AB03EBCB
:108D000086062A4656F8C81C404600F031FA35B0AF
:108D1000BDE8F08F56F823C00CFA07F0024341F883
:108D2000042B01332CFA0EF2DAE714AB2A46314653
:108D300003EB800000F01CFAD4E70FFA82FE5AF829
:108D4000C83C53F82EB034AB03EB8202013052F82A
:108D5000803C0B44BBEB030334BF012200229B4544
:108D600018BF11465CF8C82C42F82E30019B42B265
:108D70009A42E2DB731A5E42294614A85E4100F073
:108D8000EAF934AB03EB8503294653F8802C57F8F6
:108D9000803C484643EAC273013C47F8803C24B219
:108DA00000F0D9F9A8E734AB0020C6F1010C014668
:108DB00003EB860A03EB8C0CD8E730B51C4691B068
:108DC000054693F90030684600F01DF8D4F8AC3041
:108DD00069462846984711B030BD13460A46FFF74A
:108DE000ECBF70B59DF910601D463346044600F097
:108DF000CFF938B133462A4621462046BDE87040B7
:108E0000FFF746BE70BD2DE9F04F08B4F8CA04B4B0
:108E100051F8042BA3FB028940F8048B4FF0000AA1
:108E2000E4FB629A4FF0000BE5FB62AB4FF0000CE5
:108E3000E6FB62BC4FF0000EE7FB62CE51F8042B5C
:108E40004FF00008E3FB628940F8048BE4FB629A70
:108E5000E5FB62ABE6FB62BCE7FB62CE51F8042B9C
:108E60004FF00008E3FB628940F8048BE4FB629A50
:108E7000E5FB62ABE6FB62BCE7FB62CE51F8042B7C
:108E80004FF00008E3FB628940F8048BE4FB629A30
:108E9000E5FB62ABE6FB62BCE7FB62CE51F8042B5C
:108EA0004FF00008E3FB628940F8048BE4FB629A10
:108EB000E5FB62ABE6FB62BCE7FB62CE40F8049BDD
:108EC00040F804AB40F804BB40F804CB40F804EB96
:108ED0000CBC052B00F01E810C68A0F11400A1F160
:108EE0001401A2F1140252F804EB4FF0000550F8FF
:108EF000046BE4FB6E5652F804EB50F8047BE4FB81
:108F00006E6752F804EB50F8048BE4FB6E7852F86D
:108F100004EB50F8049BE4FB6E8952F804EB50F824
:108F200004ABE4FB6E9AA0F1140052F8044B51F824
:108F300004EB4FF0000CE4FB6EC540F804CB51F895
:108F400004EBE4FB6E5640F8045B51F804EBE4FBE1
:108F50006E6740F8046B51F804EBE4FB6E7840F860
:108F6000047B51F804EBE4FB6E8940F8048B51F864
:108F700004EBE4FB6E9AA0E80006062B00F0CA8022
:108F80000C68A0F11800A1F11801A2F1180252F822
:108F900004EB4FF0000550F8046BE4FB6E5652F8FA
:108FA00004EB50F8047BE4FB6E6752F804EB50F8D6
:108FB000048BE4FB6E7852F804EB50F8049BE4FB5E
:108FC0006E8952F804EB50F804ABE4FB6E9A52F849
:108FD00004EB50F804BBE4FB6EABA0F1180052F8B0
:108FE000044B51F804EB4FF0000CE4FB6EC540F865
:108FF00004CB51F804EBE4FB6E5640F8045B51F8E7
:1090000004EBE4FB6E6740F8046B51F804EBE4FBFF
:109010006E7840F8047B51F804EBE4FB6E8940F86D
:10902000048B51F804EBE4FB6E9A40F8049B51F872
:1090300004EBE4FB6EABA0E8000C072B6AD008B48D
:109040000C68A0F11C00A1F11C01A2F11C0252F855
:1090500004EB4FF0000550F8046BE4FB6E5652F839
:1090600004EB50F8047BE4FB6E6752F804EB50F815
:10907000048BE4FB6E7852F804EB50F8049BE4FB9D
:109080006E8952F804EB50F804ABE4FB6E9A52F888
:1090900004EB50F804BBE4FB6EAB52F804EB50F861
:1090A00004CBE4FB6EBCA0F11C0052F8044B51F859
:1090B00004EB4FF00003E4FB6E3540F8043B51F83D
:1090C00004EBE4FB6E5640F8045B51F804EBE4FB60
:1090D0006E6740F8046B51F804EBE4FB6E7840F8DF
:1090E000047B51F804EBE4FB6E8940F8048B51F8E3
:1090F00004EBE4FB6E9A40F8049B51F804EBE4FBAC
:109100006EAB40F804AB51F804EBE4FB6EBCA0E896
:10911000001808BCBDE8F08F013910B5024649B20D
:10912000041D0806CBB204D4013954F821000028EC
:10913000F7D0013358B250B100F18043013B52F8EF
:109140002320002322B9013803EB401000B210BDE8
:1091500052080133F6E700EB81010023884200D377
:10916000704751F8042D43EA52030B60D307F5E72B
:1091700010B500235CB2A24200DC10BD51F82340C0
:1091800040F823400133F5E7000000000000000034
:10919000C3F10803DB0070B50133002403A500BF51
:1091A0005B1920C940CAAD1B20C0184720C940CA5E
:1091B000B54120C020C940CAB54120C020C940CA1D
:1091C000B54120C020C940CAB54120C020C940CA0D
:1091D000B54120C020C940CAB54120C020C940CAFD
:1091E000B54120C06441B4FA84F0400970BD00BFAD
:1091F0004A11012350F8220001F01F0103FA01F186
:1092000008407047F0B5082289B00C460646FFF7C3
:10921000AFFFCB6A03930B6B04934B6B05938B6B84
:109220000693CB6B0793002708236A466946684676
:10923000CDE901770097FFF72BFC082305466A4626
:1092400031463046FFF724FC236B0393636B049392
:10925000A36B0593E36B0544CDE906376A46082303
:1092600069466846FFF714FC082305446A46314600
:109270003046FFF70DFC236A0093636A0193A36AEB
:109280000293A36B0693E36B0793054408236A4696
:1092900031463046CDE904770397FFF7F9FB636A5F
:1092A0000093A36AA26B0193E36A02930492636B37
:1092B000E26B0393CDE90523236A07930544082352
:1092C0006A4631463046FFF7E3FBE36A0093236BBF
:1092D0000193636B0293236A0693A36A0793054481
:1092E00008236A4631463046CDE904770397FFF7F5
:1092F0004FFF236B0093636B0193A36B0293E36BAC
:109300000393636A0693E36A07932D1A08236A4658
:1093100031463046CDE90477FFF73AFF636B00939F
:10932000A36B0193E36B0293236A0393636A049331
:10933000A36ACDE90537236B07932D1A08236A46E4
:1093400031463046FFF724FFA36B0093E36BCDE972
:109350000137636A0393A36A0493E36ACDE905378F
:10936000636B07932D1A08236A4631463046FFF790
:109370000FFF2D1A0D4C0FD435B908223146204667
:10938000FFF7BDFB01280FD00823224631463046A7
:10939000FFF7FEFE2D1AEFE708232246314630463E
:1093A000FFF776FB2D18F7D409B0F0BD20DA0200E4
:1093B00070B5036813F001060546144605D0134640
:1093C0000A460146FFF764FB064621462846FFF79A
:1093D000C2FE46B104F18042013A55F8223043F012
:1093E000004345F8223070BD2DE9F04115468AB0A2
:1093F00004460E461C22002103A8FFF729F82F1D62
:1094000095F9008003232A46314620460293FFF750
:10941000E4FC3B4602AA21462046CDF80080FFF737
:10942000E0FC2B46324621462046FFF7C6FCCDF82D
:1094300000803B4605F1840221462046FFF783FB6E
:109440000AB0BDE8F08100002DE9F041194E4FF45B
:109450008271D6F8040130B11748C268521CC2604C
:10946000304602F0D1FA00254FF4A07707EB8501D2
:109470008AB23046B258BAB189B202F0C5FA0E4883
:10948000103000EB0514204603F01EFF616819B18F
:10949000204603F09FFE07E0A16811B1204603F0CB
:1094A00099FE206800B180476D1C022DDED3BDE817
:1094B000F081000000100140D022002002F09CBB8F
:1094C00070B54FF080520024D2E94C100E2905D11E
:1094D000D2F84432694DC3F342332B60082901D0DE
:1094E0000E2908D14FF08043C3F80C41C3F8104156
:1094F000624B1B1F1C60082901D00E2955D1604BFF
:109500001B68604D2B605E4B1B1D1B682D1D2B6067
:109510005B4B08331B682D1D2B60594B0C331B68AC
:109520002D1D2B60564B10331B682D1D2B60544B8B
:1095300014331B682D1D2B60514B18331B68514D84
:1095400020352B604E4B1C331B682D1D2B604C4B64
:1095500020331B682D1D2B60494B24331B682D1DA8
:109560002B60474B28331B682D1D2B60444B2C333D
:109570001B682D1D2B60424B30331B68414D40351D
:109580002B603F4B34331B682D1D2B603C4B383315
:109590001B682D1D2B603A4B3C331B682D1D2B6027
:1095A000374B40331B682D1D2B60082904D1030065
:1095B00002D1364D344B2B60082904D1030002D16F
:1095C000334DFB232B60334B082907D1050005D110
:1095D00092F858521A6865F303021A60082904D1F8
:1095E000020002D12C4D8A012A60082901D00E29DF
:1095F00006D12A4A1568ED0702D06FF00105156003
:109600000E2903D11A6842F00F021A604FF010229F
:10961000082906D1032804D9D2F8080217491C31B9
:109620000860D2F800021E4B002803DBD2F80402C7
:1096300000280EDA012002F099FB1220C2F8000285
:1096400019680029FCD0C2F8040218680028FCD070
:109650000BE092F80C02C0070CD0012002F086FB50
:10966000C2F80C4218680028FCD0002002F07EFBF3
:1096700000F026F80C490B48086070BD3C0500401E
:109680000404001020C50040488103008C560040AF
:1096900018F50040E40E00404096024000040040EF
:1096A00000E401400090D00368230020034808B57F
:1096B000002101600068009008BD00000001014029
:1096C000BFF34F8F05480168054A01F4E06111437B
:1096D0000160BFF34F8F00BFFDE700000CED00E01D
:1096E0000400FA0502E008C8121F08C1002AFAD1D6
:1096F00070477047002001E001C1121F002AFBD112
:10970000704700000121202803DA8140054801400C
:1097100003E0402802DA2038814009B10120704777
:1097200000207047FC06FFBD800701D00020704775
:1097300001207047C3688B4206D811440069491E56
:10974000814201D8012070470020704730B585B0B4
:109750000D46164C1621ADF800101ECC0DF1040C70
:109760008CE81E00124C0221012221706270A07050
:109770000320E070217159206071FE20A0716946BC
:1097800004F109007DDF00280ED1BDF800002A4653
:10979000411CE17109212172BDF808100844ADF89F
:1097A000080001A9034872DF05B030BDD0D6020021
:1097B000A02700200823002010B586B00624182218
:1097C00008496846FEF729FE69462046FFF7BEFFB6
:1097D000002805D1044C207874DF0121207873DF44
:1097E00006B010BDE0D602000823002070B5104C72
:1097F000A66C656A01F0D8FA216B08446A1A3144F4
:10980000814200D10022082300F090FE06000DD115
:1098100001F0CAFA0022294600F0DAFBA16A81426F
:1098200003D10121A561C4E90701304670BD0000E4
:10983000383F002002F09CFB02F09AFB2DE9F84F24
:10984000254C8146924660880E46814241D80027C9
:109850004FF6FF788DF80070684600F075F82278B2
:109860006078A188884201DA401C00E00020C0B284
:10987000904204D19DF8000000F08AF827E0657856
:109880006078884201DA401C00E0002060709DF89A
:10989000000000F07DF8454519D0A068B9F1000F2F
:1098A00040F835A00DD066B16188E068324605FB0E
:1098B00001004946FEF7B1FDA06800EBC5008680B7
:1098C00002E000EBC50087800020BDE8F88F04208F
:1098D000FBE70920F9E700004823002010B50E4CF3
:1098E00003E0401C00E00020207020786178814275
:1098F00010D022786188E068A36802FB010003EBC6
:10990000C20153F83220898890472078A188884284
:10991000E9DAE6E710BD00004823002030B5CB00AF
:1099200008339DB293074FF0000401D0072030BDEB
:10993000044B9A602A44DA605C701C7058809980ED
:10994000002030BD4823002030B5EFF3108172B6FF
:109950000D4A9468012324B10370002900D162B636
:1099600030BD93604FF0E023D3F88051074C254081
:109970001560C3F88041D3F8844154605A17C3F886
:10998000842100220270E8E7AC460020FC06FFBDFF
:109990000B498A68002A11D000280FD1EFF31080FC
:1099A00072B60B684FF0E022C2F800314B68C2F883
:1099B000043100228A60002800D162B6704700009E
:1099C000AC46002070B510480146456AC06A8C6CF0
:1099D000AC2801D024B106E0486B04442D1A02E003
:1099E00001F0F6F904462A4621460848FEF739FDFB
:1099F000002807D001F052F829462046BDE8704003
:109A000001F00ABB70BD0000383F0020008002005A
:109A100030B504462C4995B04FF6FF7048800120C0
:109A20008DF812004FF65960ADF81000224604A9D7
:109A30000120A8DF002844D1244B0FCB8DE80F0074
:109A4000A11C684662DF00283BD120491C226039F6
:109A50000BA8FEF7E2FC1E4D142205F1C401A86814
:109A60001290A0788DF84A002868139006A8FEF797
:109A7000D4FC12A8069013A807902088231D06AADC
:109A80000BA9AADF00281CD11C2205F1D8010BA8C4
:109A9000FEF7C3FCE8681290A0788DF84A00686869
:109AA0001390142205F1F40106A8FEF7B6FC12A8E3
:109AB000069013A80790208804F10C0306AA0BA9AE
:109AC000AADF15B030BD000008230020A8D702008F
:109AD000A0D60200F0B585B0044614216846FEF712
:109AE000B5FC2078032308280BD12748C188491EDC
:109AF00089B2C1808288002A3ED000293CD1C28030
:109B000023702178607860228DF800208DF8011094
:109B10008DF802006078032101280AD00B2828D193
:109B200000F0B2FC8DF80300002000F0B5FC042129
:109B30001FE0207809281CD2DFE800F01B1B1B2047
:109B40001B1B051B2000D4E902706D46E91C6668EA
:109B500003F0C4FB044629193046C91C03F0BEFBC0
:109B6000044429193846C91C03F0B8FB2044C01C22
:109B7000C1B2684603F006F805B0F0BDD4E90112A1
:109B8000684602F0EEFFF2E7082300202DE9F041DD
:109B90001349034600208A68D4071ED0114CA34203
:109BA0001BD04888A0F57F43FF3B10D042F0040251
:109BB0008A60132176DF00280FD10B4EC8254FF4A1
:109BC0007A47741C3846A0476D1EFAD101E0087828
:109BD00074DFBDE8F04101F0ABBFBDE8F0810000EB
:109BE00008230020ECDA0200B0D6020038B5214C80
:109BF0000021227AD20701D0084638BDE0601E4815
:109C000000F004FE0020009001F012FA88B91B4811
:109C100013DF70B901F0B6FF58B9684601F0FAFEDB
:109C200038B96946012001F0FFFE10B9684601F01D
:109C300045FF0028E1D101F0E7FA30B1104801F00A
:109C4000D7FAA06840F00200A06000F03BFC0028BA
:109C5000D3D10B481C30FFF7DBFE0028CDD1FFF736
:109C6000ABFD0028C9D1A06840F00100A060002031
:109C700038BD000008230020F4DA02000080020052
:109C8000C027002070B50446001D2188674D86B0AE
:109C900021297CD022DC122954D018DC012977D06C
:109CA000102946D011294DD14FF6FF706880287ACF
:109CB000400704D4FFF780FD08B1FFF7BDFDE96858
:109CC00000293FD006B00220BDE8704008471329A4
:109CD0007DD0142975D01A2934D1A0E0522971D031
:109CE00016DC22292ED050292ED051292AD1A07934
:109CF000002827D021464E4802F052F9002821D0F2
:109D000006B004F10801BDE87040494802F03AB8D5
:109D1000552941D0562915D1A079002812D11321F7
:109D2000688876DF00280DD006B0BDE87040FFF7E8
:109D300083BD00886880E96809B1012088473D49F2
:109D4000688875DF06B070BD394D34F8060FA988F4
:109D50008842F7D1384800F01FFD0600F2D0628932
:109D600004F10C01FEF759FB324918227A3168469A
:109D7000FEF753FB049601956089ADF81400684620
:109D800001F08AF90028DDD031462B4801E036E0A9
:109D90003BE000F023FDD5E7E188F72913D28807DF
:109DA000B0F1404F10D0C91F89B2481EC21700EB56
:109DB000927222F00302801A081A801D81B203E019
:109DC00005E026E02BE0F7216888B5DFAAE719480F
:109DD0006A46163842F60521806A009002A8019072
:109DE0006888ADDF08B1FFF727FD00231A468521FB
:109DF00068887FDF0028A5D0FFF71EFDA2E70021BD
:109E00000091008869468FDFF4E70021688866DFEB
:109E100088E700210A4600880B4686DF82E7002398
:109E200000881A461946B1DF7CE7000008230020AD
:109E3000DC270020B6D60200F4DA0200007800F039
:109E40000100704713B90378012B01D001F0FFBA6C
:109E5000012070470022C32100F5187000F0B8B847
:109E60002DE9F043A1B00446DDE9289520200F46F6
:109E7000209098461646782102A8FEF7E7FA41217D
:109E80002046FEF7E3FAB7F8940006EB061107EB5D
:109E90008101B04201D991F8965025701DB3012D72
:109EA00004D0022D0AD0032D13D116E0002249461A
:109EB000404600F08DF8C4F8010014E020A9601CB1
:109EC000CDE900014B4642460A4902A800F094FE43
:109ED00048B1002021B0BDE8F083B1F89820601CA3
:109EE0009A31FEF79AFA4A464146204601F0AFFA07
:109EF000F0E70000C8D4020010B500284FF00000C1
:109F000006D004490870BDE81040034801F0A8B924
:109F100000F012FAC822002039A302002DE9FC410A
:109F20000646C0074FF000050ED0104F0024012256
:109F3000385D009500231146019501F0F6FC641C84
:109F4000042CF4D300F024F8B0070DD5074E0024FC
:109F5000361D0022305D032300951146019501F066
:109F6000E4FC641C042CF4D3BDE8FC81B4D40200EE
:109F70000249085C012101F0EABC0000B4D40200EF
:109F80000249085C002101F0E2BC0000B4D40200E8
:109F900010B500242046FFF7EBFF641C042CF9D316
:109FA00010BD10B543689C18446021B905E013F852
:109FB000010B01F8010B521EF9D2012010BD000067
:109FC0000249CA6B4260096C81607047383F0020CB
:109FD000F0B54FF0FF3622B11268D24300230A4D8C
:109FE0000DE03246FAE7C45C62400824D70700D08F
:109FF00037462F4087EA5202641EF7D15B1C8B4222
:10A00000F1D3D043F0BD00002083B8ED10B5044675
:10A010000068401C07D0204602F08AFE2168814279
:10A0200001D1012010BD002010BD000010B50B4C67
:10A0300090B0607800280ED100F042FE202208493E
:10A04000684600F05DFE40236A460649064800F077
:10A0500093FD0120607010B010BD00003823002077
:10A0600074D40200E4450020E0D40200F0B5146985
:10A0700006468DB020681546271DE0B1022920D084
:10A080000A2000906B4609AA304602F039FD0028EC
:10A090000FD009A901A8009A02F028FB01AE96E8AA
:10A0A0000F0005AE86E80F00236869683A4605A8E8
:10A0B00098470DB0F0BD0DB03046BDE8F04002F05D
:10A0C00089BB6946304602F01BFB0028F1D02368AB
:10A0D00069683A46684698470028EAD002980028FE
:10A0E000F5D1019870600120E3E753689B7813F085
:10A0F000C00303D0402B03D00020704700F002B80B
:10A10000FFF7B4BF2DE9FF410B46516806461446E0
:10A110008878334D00F00F0210F0300055F82250CF
:10A1200006D0102806D0202808D0302856D13EE08E
:10A1300022694DE061690120087047E0022B28D1B7
:10A14000042A26D84FF0010869463046676902F0B4
:10A15000D7FA00281AD009E00B89226903FB0022F4
:10A160006846A84770B13888401C3880029820B1F2
:10A17000616838884A899042EED3019870600298ED
:10A1800060BB02E04FF00008F7E7404604B0BDE8CE
:10A19000F081D4E904300F890288498907FB023332
:10A1A0008A421BD2521C02801A46616810E008885D
:10A1B0006169072A088009D1606801892069FEF772
:10A1C00045F960682169C06802F0B5FA22696168E2
:10A1D00004B03046AC46BDE8F04160470020D5E70A
:10A1E000F8D9020070B5204801240168C90301D5DF
:10A1F000811308E01D48016801F0F901A92904D183
:10A20000016801F0560101600024194D286A0128F7
:10A2100028D14FF4405017494068884208D123465E
:10A220004FF4805105F518706A6BFFF70BFEC8B14B
:10A2300000F0BAFD014623460F48AA69FFF702FE67
:10A2400080B14FF0A040D0F81005400E10F0010F83
:10A2500008D00648001F006800F0F900B12801D0BE
:10A26000002070BD012070BD0004004020050040AA
:10A27000383F0020DBE5B151D94100204169002978
:10A2800001D0C0680847704710B508281BD2DFE826
:10A2900000F004121A1A1A041A040120FFF73EFEF5
:10A2A0000020FFF76DFE0120FFF76AFEBDE81040B9
:10A2B0000220FFF75DBE0120FFF75AFEBDE8104007
:10A2C0000220FFF75DBE10BD10B50446801E0628B3
:10A2D00010D2DFE800F00D03030F09090A494FF41B
:10A2E000701000F0EDFA05E00120FFF705FE01E037
:10A2F00000F0DEFF05484168002903D02046BDE894
:10A300001040084710BD0000BDA50200C822002073
:10A3100010B50446062801D0072C02D1002001F018
:10A320005FF804480168002903D02046BDE81040CA
:10A33000084710BD04230020BFF34F8F0548016874
:10A34000054A01F4E06111430160BFF34F8F00BF84
:10A35000FDE700000CED00E00400FA052DE9FC41EA
:10A3600080461F4615460E4600240D4800F006FAAA
:10A3700038B11120BDE8FC8106EB043001F0F2FA9F
:10A38000641CAC42F8D1064800F0F5F9CDE900575D
:10A39000334600220221404600F02AF80020E9E777
:10A3A000582300202DE9F843104D0F4680461E46E5
:10A3B00091466946286800F0B2F9040014D01C21C7
:10A3C000FEF744F801202071C4F81490380BC4F84B
:10A3D0000080C4E902606946286800F0C1F902F013
:10A3E0006FFB0020BDE8F8830420FBE724D80200BF
:10A3F0002DE9F04387B00446DDE90E8980681D46EB
:10A4000016460F4600280BD018216846FEF71EF8A6
:10A4100002A88DF8007080E86003A168684688474C
:10A4200007B0BDE8F08330B50446006887B00D463C
:10A43000806800281FD018216846FEF707F80195AC
:10A44000A0680590207910B1012810D107E0012003
:10A450008DF8000020690290E068039005E002207A
:10A460008DF80000E06800030290606904902068A5
:10A4700081686846884707B030BD0B2803D30B3886
:10A48000C0B200F009B870470249002208780A708B
:10A490007047000020230020014908700B207047FE
:10A4A000202300200149012008707047C8220020A5
:10A4B00001490120087070470023002001237230F9
:10A4C00000F0EEBF0EB59DF8080020F00F00401C14
:10A4D00020F0F00010308DF8080068466DDF00288D
:10A4E00019D19DF80100401C8DF8010068466CDF11
:10A4F000002810D10848007A800703D50748011DBD
:10A50000806901E006A1072082B202A87CDF002852
:10A5100001D105487ADF0EBD08230020C0270020A6
:10A520004466755461726700B6D602002DE9F047A3
:10A5300081461D4616468846494502D10020BDE8A1
:10A54000F087A8EB0900040B06F6FF704FF0000A35
:10A55000070B00F0B7FAA5422AD22C4628E0A74202
:10A5600002D8BA46354601E0A246250300225146EC
:10A57000484600F017FD0028E1D1681E00F00300F6
:10A580002A1A002341464846D21C00F021FD00282B
:10A59000D5D10948A7EB0A07761B016BA9442944CA
:10A5A0000163A844002000F007FF5FEA000AC6D15B
:10A5B000002ED4D15046C2E7383F00200120FFF7DB
:10A5C0009BBC00000149416000207047F8D70200A1
:10A5D00010B50B4941600B4800F0D0F868B901F0A4
:10A5E0001DFB08491C234FF4EE7208740448A1F5C2
:10A5F000EE71001F006800F07FF8002010BD000021
:10A6000028D80200A448002002480068002800D092
:10A6100001207047582300200248007A002800D00B
:10A6200001207047A448002010B54FF44051144B4E
:10A630004C6800F500509C4204D042689A4201D117
:10A64000012200E000229C4218D144689C4215D1AE
:10A650000A78142A01D9496900E00021094A0378DF
:10A66000B1FBF2F1142B01D9406900E00020B0FBEE
:10A67000F2F0814201D0012200E00022104610BD1C
:10A68000DBE5B15140420F0070B5054608680C4645
:10A690004A6886682846314601F06EFF6068286186
:10A6A00004F10C006861B0780221B1EB901F01D178
:10A6B000241D2C6170BD000000F0D8F94FF48051CA
:10A6C000002000F011F940B90548C0F5383100F01C
:10A6D0000BF910B9034800F067F901F049FC0000DC
:10A6E0000080020089A2020010B5FDF7E0FD08B16C
:10A6F000002010BD112010BD10B531B1B2FBF3F434
:10A7000003FB14241CB1092010BD0E2010BD0160F4
:10A710000021416081608281C381084610BD70B50F
:10A720000C460546FDF778FD002802D021882868F0
:10A73000084470BD10B50A8849888A4203D1FDF7E4
:10A74000ADFD012010BD002010BD70B50C460546C2
:10A75000FDF787FD002802D061882868084470BD95
:10A7600010B50A8849888A4203D1FDF771FD01209E
:10A7700010BD002010BD002100F003B8012100F041
:10A7800006B808B56A46FDF7C4FD009808BD08B5CF
:10A790006A46FDF7B1FD08BD38B5044600258DF8C1
:10A7A00000506846FFF7D0F8216862680868904258
:10A7B0000ED9401E08600178238AE26801FB032558
:10A7C000227A2168101AC0B20A79824200D2087136
:10A7D0009DF80000FFF7DCF8284638BD38B505467F
:10A7E00000208DF800000C466846FFF7ADF8E868D9
:10A7F000298A201AB0FBF1F12A681068431C136003
:10A8000001709DF80000FFF7C3F838BD10B530B1F6
:10A81000017A42680368891AC9B21A6006E00E20FC
:10A8200010BD03681A68541C1C601170491EC9B21F
:10A83000F7D2006800210171084610BD10B54FF035
:10A84000E0224FF0FF314FF48054C2F88011C2F87B
:10A85000801200F0F9FB2046BDE81040AFF3008005
:10A8600010B504461448C0F53C3100F03DF808B17D
:10A87000FEF7E2FF00F098FA014610488069421E98
:10A88000C2F30B02801A0144002001F6FF7100F0B0
:10A890002BF808B1FEF7D0FFD4E90001002282F3C3
:10A8A000148882F3108882F3118882F3138880F36E
:10A8B0000888BDE81040084700800200383F0020AB
:10A8C00070B5084D04460E46686802F0FDFC002C89
:10A8D00006D0324621466868BDE8704002F0E6BC0A
:10A8E00070BD0000D0220020F0B50A0502D1B0F5FD
:10A8F0003C3F01D90720F0BD000B491E0C4D01243F
:10A9000000EB11332E1D0EE04209C2F1000100EBF5
:10A91000411704FA07F102D0012A03D101E02960AE
:10A9200000E03160401C9842EED90020F0BD0000EC
:10A930000006004070B5194D0024E86A243501284E
:10A9400007D0A52808D0AA2809D0AC280AD0002012
:10A9500070BDFEF74BFF0BE002F032F907E0FFF7A6
:10A9600031F805E002F02CF908B9FFF72BF80124C3
:10A97000284600F03DFA0A4900200870094800F016
:10A980001BFD08B1032070BD0120002CFBD0034942
:10A99000096A0129F7D1022070BD0000383F00206C
:10A9A00000230020B1A4020070B5284D29490026DB
:10A9B00068602748C1F80007304600F057FC18BB14
:10A9C000FFF7B8FF20B101281BD0022835D105E0E0
:10A9D0004FF47014FFF706FC10B92BE04FF4A024DD
:10A9E00000F070F81C4A20211820FEF797FF08B1EC
:10A9F000FEF722FF1948016801F0F901B12904D0DE
:10AA000007E00120FFF778FA17E0016801F04E0136
:10AA1000016000F0FFFA80B911492046FFF750FFAE
:10AA2000104800F0E1FA40B900F038F8FEF756FFA0
:10AA300041DFF9E700F0C2FB08B1032070BD2E70C2
:10AA4000094800F00DFCFFF7F9FEF6E7C8220020E8
:10AA50000C00030064000050802300201C0500400F
:10AA6000BDA50200C9A20200A5A4020010B540F6CF
:10AA7000F8700168491C02D1074900F08BFF40F6CD
:10AA8000FC700168491C05D1BDE810404FF4383115
:10AA900000F080BF10BD00000080020010B501F082
:10AAA0005DF9002803D0BDE8104002F075BC10BD70
:10AAB000034A93680A4601469860184602F0F6BBBE
:10AAC000D022002070B50E4D2878002817D101F053
:10AAD00045F9012690B10B480468A4F54864962C0A
:10AAE00000DA962402F058FC07492046FFF7E0FF01
:10AAF0004FF0E0214FF48030C1F800012E7070BD9E
:10AB00000123002004050140D5D30200406880687D
:10AB1000004710B542680830527900F0F1F8002083
:10AB200010BD2DE9F04399B01C4690460D460846ED
:10AB3000DDF88090FFF7EAFF6E6807467079A04263
:10AB400000D804462246414611A800F015F9727952
:10AB5000494601A800F0D4F801AB224611A905F13D
:10AB600008000097FDF720FE18B1002019B0BDE8DD
:10AB7000F08348F24250F9E770B516460C46054698
:10AB800000F0E2F800280ED1AA791946304600F00C
:10AB9000E8F8002807D131462046FFF7BAFF002821
:10ABA00001D10149216070BD7052464D2DE9F84335
:10ABB0000C46DDE908578146984616460D49204661
:10ABC00000F0B6F8002810D160683946407942009C
:10ABD000284600F0C6F8002807D146B14346324661
:10ABE000214648460095FFF79CFFBDE8F88348F2F0
:10ABF0001050FAE77052464D2DE9F0411D46DDE94F
:10AC000006871646044600F02DF800280DD12A4686
:10AC10003146204600F03CF8002806D13A4641462D
:10AC20002046BDE8F04100F002B8BDE8F08170B503
:10AC300015460E46044602F09FFB002807D13EB1A0
:10AC400060682968C268914205D248F2145070BD0C
:10AC500048F2135070BD83682A4631462046BDE84D
:10AC60007040184710B550B161B1416009680446A1
:10AC70008847002802D105482060002010BD48F216
:10AC8000015010BD48F2105010BD00006E524648F1
:10AC900070B515460E46044602F06EFB00280BD137
:10ACA00046B155B160682A46314643682046BDE842
:10ACB0007040184748F2105070BD002070BD000071
:10ACC0002DE9F0410B480C4D0C4F401BC6080120EC
:10ACD0003870002406E000BF55F834008047002893
:10ACE00005D1641CB442F7D3022038700020BDE8BF
:10ACF000F08100000000000000000000022300209E
:10AD000070B514460D46064600F036F8291930197C
:10AD10002246BDE8704000F02FB830B50C4605461D
:10AD200000F035F828192146BDE8304000F02FB872
:10AD300028B10068884205D048F24050704748F278
:10AD4000105070470020704728B139B10022C1E986
:10AD500000201046704748F21050704748F21350D8
:10AD6000704720B1914205D048F21150704748F227
:10AD700010507047002070470244521E04E000BF8C
:10AD800011F8013B02F801398242F9D270470144BF
:10AD9000491E05E002780B7800F8013B01F8012913
:10ADA0008142F7D2704700004FF44050074A416893
:10ADB000914207D18068411EC1F30B01401A00F691
:10ADC000FF7070474FF4805070470000DBE5B151D1
:10ADD00000B5FFF7E9FF054989690A18401E0844D4
:10ADE000C0F30B00101A00F6FF7000BD383F0020C2
:10ADF00000210160416081600148016370470000EB
:10AE0000383F00202DE9F0419846214F16460C4668
:10AE10000546002301215BB1012B11D0022B1ED06E
:10AE20000020381AA0F50050A8421BD201221AE0D7
:10AE3000FFF7CEFF8EB11749096A0129F1D00CE066
:10AE4000FFF7B2FFB8F1000F05D14FF44051124A9D
:10AE50004968914201D00121E3E70021E1E74FF485
:10AE60008050DEE7002242EA0400884305D0022B2E
:10AE700003D25B1CDBB2022BCCD912B10420BDE89B
:10AE8000F0811BB103481830FFF7B2FF0020F6E74E
:10AE900000800200383F0020DBE5B15170B5044668
:10AEA0000078092811D2DFE800F0100510112510F4
:10AEB000381013000D461D490320C9688847606992
:10AEC00000F056FBFFF7D9FA687070BD084628E01D
:10AED0000D46A18A206900F027FBFFF7CEFA6870C3
:10AEE0002846FFF76DF8E1680029EED02069BDE83B
:10AEF000704008470C460D490831081F00F052FB0E
:10AF0000FFF7BBFA60700128DFD1002000F054FA8F
:10AF10000028DAD00A20607070BD08464FF4007136
:10AF2000C160BDE87040FFF74BB80000242300204B
:10AF300070B51A4A05780124936C092D2CD2DFE8EC
:10AF400005F02B052B0B0F2B252B080000F054FFD1
:10AF500022E000F0C7FF1FE08B60106D48601BE02F
:10AF6000D2E91454566C2C1BA64203D0082048701A
:10AF7000012411E00024556554642146D36400F097
:10AF800075FF07490420C968884705E08B60106D8C
:10AF900048604FF48050C860204670BD383F0020A4
:10AFA0002423002013460A460146014800F0F0BB66
:10AFB0006C23002008B1034900E003490022034844
:10AFC00000F0FCBB34D8020004D802006C2300203F
:10AFD00008B5009313460A460146024800F086FC75
:10AFE00008BD00006C230020084910B5086000204F
:10AFF000FFF78EF9064800F00DFA002804D1BDE8ED
:10B000001040034800F026B810BD000004230020C3
:10B0100011A30200002070471FB58908002201AB70
:10B02000009283E80700684618DF04B010BD0000F6
:10B030001FB5044B0FCB8DE80F00684618DF04B036
:10B0400010BD0000B8D702004FF4805041040860E2
:10B050000020704710B5040011D00120FFF7AAFFAF
:10B0600000280BD100F04EFA00F0DEFA48B1094991
:10B07000081F00F097FA012803D0032010BD072015
:10B0800010BD04480838C4600020FFF705FA00200E
:10B0900010BD00002C230020816819B1024A18213C
:10B0A000FEF7CCBB07207047ADB00200AFF30080C5
:10B0B00030B587B0044618221F496846FDF7ADF940
:10B0C00020788DF8000022781C4D0D2A25D2DFE86B
:10B0D00002F0240B270B0B240B240B242424070041
:10B0E000E968072088471BE020466946062A01D008
:10B0F000012A01D1027C2A702A78012A05D0022A6D
:10B1000006D000202870052008E0FFF7C7FE07E002
:10B11000FFF70EFF20B907B030BD02208DF8010007
:10B12000D4E90112684690479DF801000128F2D049
:10B13000E96805208847EEE7E0D7020024230020D5
:10B1400038B10549016005494160012101720020C3
:10B1500070470E207047000061B1020099B10200F3
:10B1600010B50C0001464FF0110007D02278052AD7
:10B1700005D2DFE802F00F050D0F0F000E2010BD05
:10B18000084600F051F80028F9D10221217010BDC5
:10B19000112010BD082010BD0246082041B10B78D7
:10B1A000022B04D1022A05D0032A00D111207047B6
:10B1B0000E207047002003220A70704770B50B48BC
:10B1C0000024D0F82413491C03D1D0F86403401C98
:10B1D00009D04FF43C35284600F0C4FBC92203498E
:10B1E000284600F0EFFB204670BD0000383F0020ED
:10B1F00010B528B11C220349FDF70FF9002010BD3E
:10B200000E2010BD64F3020010B5064C0022182178
:10B21000201DFEF7DDFE2168814201D1012010BD15
:10B22000002010BD64F3020070B50C4D0400D5F889
:10B23000640305F5597503D0401C03D0082070BD88
:10B240000E2070BD00221821201DFEF7C1FE2060D7
:10B2500007222146284629DF70BD000000F00200C9
:10B26000014901F05BBD000000F0020010B5FFF7DE
:10B27000A1FE30B900F01CF8002000F09DF8002875
:10B2800000D0032010BD000010B5FF224FF4007164
:10B290000648FDF7D4F8054820212438FDF7D6F8F4
:10B2A000024900205C39086310BD0000943F002073
:10B2B0002DE9F0472E48FEF7A9FE2E4E07463468CA
:10B2C0002046FEF7A3FE4FF0010A4FF0000958B1E7
:10B2D0006068012806D02046FEF7BCFDD4F85C1259
:10B2E000884201D1012500E00025234C4FF00208DF
:10B2F0004FF460719FB10A461D492046FDF78DF855
:10B300009DB1366825465422311D281DFDF785F86C
:10B310004FF4327206F15C0105F15C0003E015B3F5
:10B320000A4615483168FDF778F86068012818D199
:10B330001249402201F5E470FDF76FF80F491C2215
:10B34000403101F5E470FDF768F884F8609284F804
:10B35000A1A20B4884F8E292E169C0F82210C4F877
:10B360000480BDE8F0870448FDF770F8F7E70000B7
:10B3700000F0020034230020383F002094400020D9
:10B38000B841002070B50546094801F0D1FC084CD1
:10B3900020602046FEF75EFDC4F85C02A4F5E06381
:10B3A0002A462146BDE87040024801F0C6BC0000B4
:10B3B000383F002000F0020070B505460020FFF77E
:10B3C000E1FF040003D10349284601F0A7FC204611
:10B3D00070BD0000383F00204FF4805070470000DF
:10B3E0002DE9F04107460948094D401BC6080020D9
:10B3F000044607E005EBC40041683846884700284A
:10B4000002D1641CB442F5D3BDE8F081F4DA020045
:10B41000ECDA02002DE9F04107460948094D401BCE
:10B42000C6080020044606E055F834103846884720
:10B43000002802D1641CB442F6D3BDE8F0810000BC
:10B44000F4DA0200ECDA0200012201F0F1B938B5B9
:10B45000144602780B467AB1012A04D0022A0DD094
:10B46000032A1BD112E0D0F80150002221461846D1
:10B47000FEF7AEFDA84211D1012038BD01B0224631
:10B48000BDE830400023401C00F00AB8411C4022B7
:10B490000020009400F0F2F80128EED0002038BD22
:10B4A0002DE9F041AAB005462020884628901E4686
:10B4B00017460124782102A8FCF7C8FFFEF7B6FD65
:10B4C0002EB12022294620A8FFF756FC20AD28A93E
:10B4D0000A48CDE900013B464246094902A8FFF768
:10B4E0008BFB28B9202229460448FCF7BAFF00B19B
:10B4F00000242AB02046BDE8F08100008C460020E0
:10B50000C8D4020010B50648064C806B20B101F08B
:10B51000FDFD08B1012000E00020207010BD0000FA
:10B52000383F0020382300202DE9F0410F4C07461A
:10B530000D46E06BA26B01264119914201D9032609
:10B5400010E00A492A465C3108443946FCF765FF99
:10B55000E06B064A2844E063403229463846FEF74D
:10B5600037FD20643046BDE8F0810000383F002000
:10B5700070B504004FF0010504D0B4F5007F03D985
:10B58000042508E0032506E0044900200870FFF7C1
:10B590007BFE03488463284670BD000038230020EA
:10B5A000383F00202DE9F04106461D480F46C16B8B
:10B5B000806B814201D008242FE01A4D287840B1D9
:10B5C000FFF706FC30603946E86801F0A9FE044642
:10B5D00023E001F09BFDF8B100F02CF804460020B8
:10B5E00030603860012C0FD13946E86801F098FED0
:10B5F0000446012808D13868012700213B460A4645
:10B60000FFF700FC18B10424FFF73EFE05E0FFF74A
:10B61000DFFB30602F7000E005242046BDE8F0819C
:10B62000383F002038230020014800787047000090
:10B630003823002038B50F4C251D002094F86C31BC
:10B64000014602463BB194F8D802B4F8DA2204F578
:10B65000B87504F53771084B9C6800945B6800F07E
:10B660000DF8012804D1281DBDE8384000F050B87D
:10B6700038BD0000B8420020382300202DE9F041F9
:10B68000A2B0064620200D4620901F461446DDF845
:10B69000A080782102A8FCF7D9FE00202190FEF7B7
:10B6A000C5FC25B12EB1162022B0BDE8F0811320D3
:10B6B000FAE720A91448CDE9000143463A46134968
:10B6C00002A8FFF799FA08B9402C01D00A20EBE74D
:10B6D0000D48224629464038FCF79FFE0A482021A3
:10B6E0004038FFF71AFB084840214038CDE90001F7
:10B6F000A0F14801044A21A8209BFFF757FA08B19E
:10B700000520D1E70120CFE76C460020C8D4020015
:10B7100070B5044690F85400012570B394F85500B4
:10B7200028B1012803D0022801D003282AD194F897
:10B730006E00032801D0142525E0207AE8B1E068E6
:10B74000342801D011251EE0204601F085FA68B1A9
:10B75000207898B194F855100C4849B1012907D0C8
:10B760006168C06881420ED810250CE012250AE0FD
:10B7700061688068814206D2F6E703E094F85500DC
:10B78000012800D00F25284670BD0000383F00205A
:10B790002DE9F0410446406815461E4602680F46F2
:10B7A0006A432046FDF7C6FF206833462A46D0F894
:10B7B00010C039462046BDE8F041604701600B6883
:10B7C000114618472DE9F04128B1016819B1C9693E
:10B7D000BDE8F04108470D4D0D480024461B1427D5
:10B7E0000DE000BF04EB840005EB8000016829B187
:10B7F000C969884710B10120BDE8F081641CB6FB1F
:10B80000F7F0A042EED80020F6E700006C230020FD
:10B8100080230020044801214174007A08B10020EF
:10B820007047012070470000A4480020012801D083
:10B83000032808D10449002201284A7400D00020BE
:10B84000087401F0EFB87047A448002070B50146B5
:10B85000022801D0032943D1224C207A00283FD06E
:10B86000012831D002282FD11F4800230229006867
:10B8700002D0032928D119E0E360027912B1012A2C
:10B8800022D10BE0D0E90565721B142A00D31422E3
:10B890002A4482614569AA420ED015E00169491C1B
:10B8A0000161426991420FD1237213E0E268521C98
:10B8B000E260082A08D9E360237202290AD00D2128
:10B8C000FEF7B1FD01F0A4F8607C28B1BDE870403E
:10B8D00000F0AAB90021F3E7BDE8704001F0A2B87A
:10B8E00070BD0000A44800205C2300202DE9F8432F
:10B8F00004461D4616460F460846DDF82080FDF733
:10B9000013FF3046FDF710FF2A4639462046FDF763
:10B9100011FFCDF8008020682B463246D0F80CC0CD
:10B9200039462046E047BDE8F88370B541EA420158
:10B93000DDE904564FF0A04441EA830141EA0521C4
:10B9400004EB800041EA0641C0F8001770BD0122F7
:10B950004FF0A043824011B1C3F808257047C3F8E7
:10B960000C257047094902220A60BFF36F8FBFF3AD
:10B970004F8F0A1D106006480268002AFCD0002084
:10B980000860BFF36F8FBFF34F8F704704E501402E
:10B9900000E40140094A01231360BFF36F8FBFF336
:10B9A0004F8F0160064801680029FCD0002010601C
:10B9B000BFF36F8FBFF34F8F7047000004E5014066
:10B9C00000E4014070B50E4C01232360BFF36F8F7C
:10B9D000BFF34F8F00230B4D08E000BF51F82360E9
:10B9E00040F823602E68002EFCD05B1C9342F5D3F8
:10B9F00000202060BFF36F8FBFF34F8F70BD00003A
:10BA000004E5014000E4014008B5002242504058DE
:10BA1000009008BD20B1034909680160002070470B
:10BA20000E207047CCD90200FEB506460C460846EB
:10BA3000FFF7F0FF002840D1002500950195012770
:10BA400006208DF80060ADF8040002958DF80270B4
:10BA500069462020226869DF0095019502958DF8DE
:10BA6000017069464020226869DF00958DF800600A
:10BA7000F720ADF80200019502956946232022685F
:10BA800069DF0095019502958DF8007069460120E7
:10BA9000226869DF4FF4B060009001950295694615
:10BAA000A120226869DF0095019502958DF800506C
:10BAB0006946A020226869DF0020FEBD60DF002803
:10BAC00002D1024A01211170704700006723002053
:10BAD00030B51548ADF5017D0078002821D04FF430
:10BAE000FA7500BFADF8005280A9684661DF38B131
:10BAF000052816D00DF5017DBDE83040FDF79CBE50
:10BB00006C460A497DA800F0BBF806E0D0E90021A8
:10BB1000204690477DA800F0CAF87F980028E1D021
:10BB2000F4E70DF5017D30BD67230020D0D9020078
:10BB3000F8B5134C2078C0B10120A07001F0C0F816
:10BB4000112814D0022001F0D3F800258DF8005000
:10BB50006846FDF7F9FE11DF064625709DF80000E6
:10BB6000FDF716FF2EB13046F8BD0820F8BD0020C5
:10BB7000F8BDA57001F07EFA032001F0B9F8F6E7F0
:10BB8000642300207CB5194C207808B108207CBDC6
:10BB90000120A070002001F093F8112819D0002096
:10BBA00001F0A6F812480026006801908DF80060A8
:10BBB0006846FDF7C9FE0F4901A810DF05000AD04D
:10BBC000002020709DF80000FDF7E2FE2DB1284610
:10BBD0007CBD00207CBD0120F3E7A670667001F0FB
:10BBE00069FA012001F084F8F3E7000064230020E3
:10BBF00064D90200359802000EB50749684600F086
:10BC00003FF805E0D0E900108847684600F04FF89B
:10BC100002980028F6D10EBD80D9020001480078B4
:10BC200070470000642300200548817819B100782E
:10BC300018B1FFF77DBF08207047FFF7A3BF0000D2
:10BC4000642300201FB568464BDF30B1052814D0AF
:10BC500004B0BDE81040FDF7EFBD084901A800F0B1
:10BC60000FF806E0D0E900210098904701A800F005
:10BC70001EF803980028E6D0F4E71FBDECD90200B7
:10BC8000016009684160AFF3008010B5D0E9002180
:10BC90005368994201D1002104E0D1E90034A34264
:10BCA00002D01946816010BD08314160F0E781681B
:10BCB00000290BD0026892680A44826041684B6890
:10BCC0009A4203D108314160FFF7DFBF704700009F
:10BCD0002DE9F04104461348134BC01A0C21B0FB68
:10BCE000F1F6A0694FF0FF3110F8022C02B921697A
:10BCF000002011E000EB400503EB85052F6897421B
:10BD000009D14F1C02D06F688F4204D194E80F0014
:10BD1000AD68A84703E0401CB042EBD3012020608F
:10BD2000BDE8F08144DB020038DB020010B51446A8
:10BD300012680830202A02D248F2145010BD0022A6
:10BD400001F023F80028F9D120202060002010BD48
:10BD5000083001F0A3B8083001F062B90248006869
:10BD6000002800D00120704700040140034908600A
:10BD7000034801680029FCD07047000004E5014039
:10BD800000E4014030B587B00C460546182217493B
:10BD90006846FCF742FB217B15488DF800100195A1
:10BDA000012906D0022917D0062919D1607B0490F9
:10BDB00016E08188C180607B0490217CE08961F37A
:10BDC0001F40617C40EA016005900498012807D17A
:10BDD0000848FFF705FB03E0B4F80D108180C1802F
:10BDE0006846FFF759F907B030BD000008D70200D8
:10BDF00008230020ECDA02002DE9F0410C4605464C
:10BE0000FFF712FC0826B8B16969032041B3154A4F
:10BE1000154B0F0505D0576DD3F808C00F44674583
:10BE20001ED1B1F5805F01D9042019E0506DD3F81F
:10BE300008C04718674502D96670BDE8F0815164B3
:10BE4000D16C10659164106369695A6801F6FF71DD
:10BE50001044090B0022FFF7A5F80028EDD00520BB
:10BE60006070EAE7383F00202423002010B5044624
:10BE700086B00020FFF7A6FC30B1154A18212046F5
:10BE8000FDF7DCFC06B010BD182212496846FCF72D
:10BE9000C4FA1148026D114881688A4210D1406885
:10BEA000FFF7D2FA8DF80100FEF7E7FA8DF80100EE
:10BEB000D4E90112684690470948FFF77DFAE1E7A7
:10BEC00001208DF80100D4E9011268469047D9E7B6
:10BED0006DBE0200C8D70200383F00202423002096
:10BEE00065BF02002DE9F0410E460446FFF79CFBBA
:10BEF00060B11A4DD5E91401401AA18A6A6C084450
:10BF0000904205D903207070BDE8F0810820FAE75F
:10BF1000134A286B52688718104A20694832FEF786
:10BF200057F8D4E903318046A28A3846FFF750F823
:10BF300020B1D4E90310BDE8F0410847A18A286B7D
:10BF400008442863A18A286DC5F8488008442865FC
:10BF5000C6F80880286D7060D6E70000383F0020E2
:10BF60002423002001490620C96808472423002013
:10BF7000BFF34F8F05480168054A01F4E0611143A2
:10BF80000160BFF34F8F00BFFDE700000CED00E044
:10BF90000400FA0501460148FEF720BCF4DA02006D
:10BFA00030B58A1D8B79083187B0022B33D1538885
:10BFB0008489A3422FD1127A012A2CD1184C0DF179
:10BFC000040C3CCC8CE83C000A89ADF80C204A8972
:10BFD0000C3104911249ADF80E208039114C096AD8
:10BFE0000591CDF818D0018A05AA6088ADDF18B98F
:10BFF0006846FDF723FF38B10020ADF8080001A91D
:10C000006088B0DF50B106E040F2FD10ADF80800E6
:10C0100001A96088B0DF002007B030BD0120FBE738
:10C0200020D7020008230020F8B50D461446064626
:10C03000694600F05DFA00280FD0009BB3F5803F01
:10C040000AD2981C834207D8A9780222B2EB911F2A
:10C0500002D02989814201D20020F8BD2380A11C91
:10C060003046009A00F07AFBF8BD114600F0D5B8D2
:10C07000114600F0E7B8F8B50C4615460646694685
:10C0800000F036FA00280CD0009A501C904207D3DA
:10C09000A1780223B3EB911F02D02189814201D202
:10C0A0000020F8BD2946304600F058FB009A0021D8
:10C0B000A954F8BD2DE9FF410C46CE681746054648
:10C0C000694600F01DFB00280ED0E06800280BD068
:10C0D000A0783A46C0F3011002283146684606D0DF
:10C0E00000F0DEF80199696004B0BDE8F08100F06D
:10C0F00085F8F7E77CB50D461446694600F095F9DA
:10C10000002820D02889082806D0042809D0022831
:10C110000AD001280CD015E0DDE90001C4E90001D6
:10C120000AE00098206006E0009800B2208002E05B
:10C13000009840B22070C117DDE9002350405940FB
:10C14000084301D000207CBD01207CBD7CB50D469C
:10C150001446694600F0A7F9002820D0288908284D
:10C1600007D00021042809D002280AD001280CD0C9
:10C1700014E0DDE90001C4E9000109E00098206055
:10C1800006E0009880B2208002E00098C0B22070E3
:10C19000DDE9002350405940084301D000207CBD18
:10C1A00001207CBD7CB50D461446694600F07BF944
:10C1B000002820D02889082808D00099CA17042808
:10C1C0000BD002280CD001280DD013E0DDE90012BD
:10C1D000C4E900120846134608E00846216004E05E
:10C1E00008B2208001E048B22070C3174840534095
:10C1F000184301D000207CBD01207CBD70B50D46E8
:10C20000064614461146284600F095FA224629466D
:10C210003046BDE8704000F043B838B50C46042203
:10C22000694600F09BFA00280BD09DF80210BDF87B
:10C23000000061F31F409DF8031040EA0160206098
:10C24000012038BD1CB50C460822694600F086FA6C
:10C25000002824D09DF801109DF800209DF80230A0
:10C26000080E42EA012242EA034240EA13409DF8E6
:10C2700003309DF8041040EA132008439DF8051090
:10C2800042EA036240EA01209DF8061040EA0140BC
:10C290009DF8071040EA0160C4E9002001201CBDA0
:10C2A0002DE9F04F05469DB000200F9006461090F6
:10C2B0004FF0FF3A01A800F05FF94FF0010B0DF1CC
:10C2C0003C0983E012AB6A460BA9284600F0CAF885
:10C2D00050B101A8009900F060F960B1029880782F
:10C2E00010F0300F54D061E09DF84800002871D163
:10C2F0001DB0BDE8F08F0098B04243D3029C01AE60
:10C300000298807800F00F00082812D0304600F024
:10C310005BF90298A042F3D156460098B04231D35F
:10C32000D5F8088007909DF82C000E9005980468B9
:10C3300021E002980688F0E7206807682FB12146BF
:10C3400028460E9B079AB84712E011952168079876
:10C350000E9F8968098881420CD1214617A8FEF7F3
:10C3600093F984F80CB017AA39461198FDF7BDFE71
:10C370000028BDD0A46814B1A9684145DCD0A968E3
:10C38000414523D19DF82C10284600F023FA1BE0EC
:10C39000039840280AD200F01F000BFA00F203981D
:10C3A000400959F82030134349F82030EC682CB18B
:10C3B00001AB9DF82C2028460099A04701AA9DF8C2
:10C3C0002C102846FDF791FE002891D0A86800287F
:10C3D0007FF478AFDDE90204857801A800F0F4F875
:10C3E0000028F7D115F0300F03D10298008800B172
:10C3F000641CC4B10020494605E000BF51F820206C
:10C40000521C0ED1401CB0EB541FF7D3600959F8F1
:10C41000201004F01F00C0F120022AFA02F081422D
:10C4200001D0002064E7012062E71CB50C46694694
:10C4300000F039F8002814D0DDE90002C10709D066
:10C4400051084FEA30006FEA00026FEA0100C4E9C8
:10C45000002004E051084FEA3000C4E900014FF029
:10C4600001001CBDF8B507460020187008700E4684
:10C4700010601C4615466946384600F039F8010040
:10C480004FF0010009D0009959B1C8082860009800
:10C4900000F0070030700120F8BDB96809B1002034
:10C4A000F8BD2070FBE72DE9F84300268846814659
:10C4B0003446354604E0402E02D30020BDE8F88320
:10C4C0006946484600F076F90028F7D09DF80070DC
:10C4D000324607F07F00C10FFBF790FF294304436A
:10C4E000F61D0D463806E6D4C8E900410120E5E70F
:10C4F000F8B50E460746694600F05CF900280AD0F8
:10C500009DF80040200616D5072504F07F0403E0BF
:10C51000202D01D30020F8BD6946384600F04AF9C5
:10C520000028F8D09DF8001001F07F00A8400443D7
:10C53000ED1D0806ECD401203460F8BD10B5596833
:10C540000B4AC968914212D10A4AD0E90110D2E9D6
:10C550000134234301D0002008E011F8013BA0F191
:10C5600001001B06F9D4C2E901100120907010BD32
:10C5700050D5020038230020C26000230160C0E9CA
:10C5800001138B881A440261B1F906301A444261E2
:10C590000888002800D00120704770B545680E4615
:10C5A000044660680188B14206D1807800F00F002F
:10C5B000082801D0012070BD204600F005F8606811
:10C5C000A842EED1002070BD30B541680A885AB14A
:10C5D00001F1100343600A8A42B18C780A89C4F3DE
:10C5E0000115032D07D00BE0002030BDC2680168A3
:10C5F000FFF7C2FFF8E79D78C5F30115032D06D0BC
:10C600000225B5EB141F08D14C89624309E08D88DF
:10C6100004690022641B046103E0B5EB941F00D1A0
:10C620000422897811F0300F02D18168491C8160A1
:10C630009C880169214411440161B3F90620114429
:10C640004161012030BD30B54168002487B0897850
:10C6500001F00F02082A11D08A091ED00222B2EB83
:10C66000911F09D10269C1F301110229146001D09F
:10C67000032901D14069048007B030BD0069056815
:10C6800008E02C7329466846FDF7FEFF6846FFF771
:10C69000DAFFAD68002DF4D1EEE7C1F301110129F5
:10C6A00012D00229E6D00329E4D04268917801F043
:10C6B0000F0107290BD0D16881B11289006907B039
:10C6C000BDE83040FBF7A9BE41690C70EDE7016998
:10C6D000D06807B0BDE8304000F02DB8118900697E
:10C6E00007B0BDE83040FBF7B1BE000010B5034B0A
:10C6F000002408C080E8160010BD0000A39F0200BF
:10C7000038B50D4604466946FFF7F2FE00280BD007
:10C71000D4E90002D4E90213C5E90002C5E9021315
:10C720000098814201D2002038BDA860A168081A93
:10C73000A060012038BD00B50A4687B001466846B2
:10C74000FFF71AFF002807D06846FFF77CFF68460E
:10C75000FFF73AFF0028F7D107B000BD7FB51446B8
:10C760000546A9B9124A2868904208D110E0102263
:10C7700069462846FFF7F2FF002807D0103C102C2E
:10C78000F5D8224669462846FFF7E8FF04B070BD99
:10C79000A868A04201D20020F8E72B68224628466C
:10C7A00098470028F2D0A868001BA8600120EDE798
:10C7B000A39F020010B504468068002809D02368B2
:10C7C000012220469847002803D0A068401EA060A0
:10C7D000012010BD38B5002439B1012912D0022939
:10C7E00012D005291DD0002038BD0546012269461A
:10C7F0002846FFF7B3FF90B19DF800000006F5D47E
:10C80000012038BD08220DE005466946FFF770FE9D
:10C8100028B100212846009AFFF7A0FF38BD204626
:10C8200038BD0422BDE838400021FFF797BF000063
:10C830002DE9F04F81462C4817460E46C5680A463A
:10C8400093B0012449462846FDF738FEDFF89C8066
:10C85000A24670B195F8550068B100F00101C0F32F
:10C8600040024B462846CDE9006700F043F8D8B1B6
:10C870001BE0172419E0CDE9006A4B460022294647
:10C8800002A8FDF7EDFA4FF0000B68B10FB341229B
:10C8900002A91748FBF7C1FDC8F820B0C8F82CA0C2
:10C8A0006968C8F8081017E005246FB1012C13D08F
:10C8B0000E482430FEF79CFAFEF7E6FCC8F84890D4
:10C8C00013B02046BDE8F08F012C02D0FEF7DCFC4F
:10C8D000F6E7C8F814A0F3E7002231464846FDF712
:10C8E00077FBC8E90960E7E738230020383F0020DC
:10C8F000D94100202DE9F047A4B08946DDE92C5A42
:10C90000044698461646442102A8FBF79FFD4421A1
:10C9100013A8FBF79BFD4746B9F1000F38D008F587
:10C920000050384A4368A16D934255D14B1EC3F362
:10C930000B03C91A41F6FF73D0F808C019448C459F
:10C940004AD34FF440514B6893420DD10A78102AD4
:10C9500001D9096900E000210278102A01D9006993
:10C9600000E00020814237D14046FDF75DFE00B176
:10C970008EB30121A06DCDE900014346002221467E
:10C9800002A8FDF76DFA002827D0A06D07442D1AE4
:10C9900056B10020CDE900503B464A46214613A837
:10C9A000FDF75EFA002818D0BAF1000F28D0164D16
:10C9B000B9F1000F19D04046FDF736FE18B105F168
:10C9C0001800FEF715FA412202A91048FBF725FDD1
:10C9D00036B1AC2005E0FFE7002024B0BDE8F087C9
:10C9E000A520E862A06D686301E0AA20E8623EB17C
:10C9F0000648412213A98230FBF70FFD6068E8600A
:10CA00000120EAE7DBE5B151383F002098410020E2
:10CA1000034802490068FDF78DBE00006023002036
:10CA200024D802002DE9F041224C0025224E207A24
:10CA3000012730B92148311D0068FDF786FE3060BE
:10CA400038B1022020723168087928B101281CD140
:10CA500014E06560BDE8F081D1E90503C01A14282F
:10CA600000D31420B7EB900F01D2820800E001221E
:10CA70000869C9681844194429DF03E0D1E90301B2
:10CA8000084428DF58B1112812D003213068FDF77F
:10CA9000CAFC25726560BDE8F041FFF7B9BF207C94
:10CAA0000028D7D1BDE8F04100210220FEF7CEBE1C
:10CAB0002772CFE7A44800205C23002024D802007E
:10CAC00010B5074C201DFDF759FE002806D1607CEB
:10CAD000002803D1BDE81040FFF7A4BF10BD00003F
:10CAE000A448002010B510461A46FBF796FC00201B
:10CAF00010BD10B510461A46FBF78FFC002010BD84
:10CB00002DE9F0411E681C461546074621B1012952
:10CB100018D0052923D119E000202060401C206096
:10CB2000B0421CD8012229463846FFF717FE0028DC
:10CB300006D015F8010B000601D52068EEE70120AC
:10CB4000BDE8F08108200246186002E00420024699
:10CB5000186029463846BDE8F041FFF7FFBD0020C8
:10CB6000EEE770B516460A460446C11C104600F0B2
:10CB7000B5FB054661193046C91C00F0AFFB2844DF
:10CB800070BD000003B5094A85B0D2E91612CDE99F
:10CB9000001207498989ADF8001006A9CDE90210F5
:10CBA000044869464088AEDF07B000BDA0D6020049
:10CBB000DC270020082300200846704708467047FD
:10CBC00070B5FEF709FC114A114E136B546B916C52
:10CBD000E21A551EC5F30B05521B42F20405184418
:10CBE0006D5802F6FF72B54201D0032070BD1944A2
:10CBF000A34201D1002070BD0823FDF797FC002857
:10CC0000F9D1BDE87040FEF7D7BB0000383F0020E7
:10CC1000DBE5B151F0B50546002003464FF4405422
:10CC20000C4E4FF6FE7712E0D4F804C0B44505D19F
:10CC300055F823C0B4F80CE0F44504D02AB155F8F7
:10CC400023C0BC4501D10120F0BD5B1CDBB28B428F
:10CC5000EAD3F0BDDBE5B15110B54FF44051174BAD
:10CC60004A68018A9A4221D171B100F114034269E4
:10CC700090F8550062B1042808D00022BDE81040A9
:10CC8000C9B21846FFF7C6BF002010BD0122F5E764
:10CC900010B1012808D1F7E7012905D9C9B200224E
:10CCA0001846FFF7B7FFEFE7012010BD11B141694A
:10CCB0000029E9D100780028F6D110BDDBE5B1519B
:10CCC0003EB5044609496846FEF7DAFF08E000BFB2
:10CCD000D0E900212046904730B16846FEF7E7FFD3
:10CCE00002980028F4D13EBD11203EBD68D9020053
:10CCF0003EB5044608496846FEF7C2FF07E000BF9C
:10CD0000D0E90021204690476846FEF7D0FF029800
:10CD10000028F5D13EBD000074D902000246034848
:10CD2000014B006800F009B8B83B00203423002014
:10CD300000225821001DFDF74BB92DE9F0411446A2
:10CD40004FF460751E460F4680462A46FBF789FB66
:10CD500030B1002201214046FEF724F998B905E0E0
:10CD60000CB10020A0470020BDE8F0812A463946DA
:10CD70003046FBF752FB23462A4631464046FEF733
:10CD800027F90028F0D00320EEE770B516460D46CF
:10CD9000040007D035B1206C8022002138282254AD
:10CDA00003D307E00E2070BD2154401C3828FBD36C
:10CDB0000BE02154401C4028FBD32146084600F0DC
:10CDC00097F838212046FBF741FB216CD4E912305B
:10CDD0004A0FC900383459185041C4E90410227C64
:10CDE000E2710A0A42EA0062A2710A0C42EA0042B7
:10CDF0006271020242EA116020716069E070010A0A
:10CE0000A170010C6170000E04F838092146084633
:10CE100000F06EF84FF00002EEB1E06ED100C840B5
:10CE2000A854A36ECB40A8180371636ECB40037265
:10CE3000236ECB400373E36DCB400374A36DCB40F3
:10CE40000375636DCB400376236DCB40521C037793
:10CE5000042AE2D31FE018235042216D03EBC000E7
:10CE6000C140A954666DC640A9180E71A66DC64092
:10CE70000E72E66DC6400E73266EC6400E74666E68
:10CE8000C6400E75A66EC6400E76E66EC640521CB3
:10CE90000E77042AE0D3002070BD0000A8B1002165
:10CEA0000164C0E912110A4901650A4941650A494C
:10CEB00081650A49C1650A4901660A4941660A490C
:10CEC00081660A49C166002070470E207047000045
:10CED00067E6096A85AE67BB72F36E3C3AF54FA50B
:10CEE0007F520E518C68059BABD9831F19CDE05B37
:10CEF0002DE9F04FC8B0002213466F46CC181B1D19
:10CF00002588A6786DBA2D04E47845EA06252543E0
:10CF100047F82250521C102AF0D31BE007EB820185
:10CF200051F8083C4FEA734484EAF34484EA9324BA
:10CF300051F83C3C4FEAF31585EAB34585EAD30343
:10CF4000234451F81C4C51F8401C2144194447F823
:10CF50002210521C402AE1D3036D4793416D469144
:10CF6000846D4594C26D44929246026E4392456E22
:10CF70004295A946856E4195C66E4096B3460026F9
:10CF80004FEAB21787EAF22787EA726C02EA0907CA
:10CF900025EA020887EA0807BC44204F57F8268094
:10CFA00008EB0B07BC445DF82670AB460CEB070E94
:10CFB0004FEAB30787EA733787EAB35C81EA04076D
:10CFC0004D4601EA040891461F400AEB0E02A246B4
:10CFD00087EA08070C46BC441946761C0EEB0C0386
:10CFE000402ECDD3479E33440365469B194441658B
:10CFF00045992144816544995144C165439911443F
:10D0000001664299494441664199294481664099A3
:10D010005944C16648B0BDE8F08F000054D8020002
:10D020002DE9F04116460F46040004D006B317B1AF
:10D030000025A8461AE00E20BDE8F081216C785D3D
:10D040006054206C401C206440280ED121460846C4
:10D05000FFF74EFFD4E912014FF40072801841F13E
:10D060000001C4F84080C4E912016D1CB542E5D34B
:10D070000020E1E710B51620FCF744FB48B10C484E
:10D0800082684FF4800152B1016821F4800101608F
:10D0900010BDBDE8104042F20100FCF7CDBB4FF0DF
:10D0A000E020C0F88011BFF34F8FBFF36F8F10BD2A
:10D0B000AC46002010B51620FCF724FBA0B11148A7
:10D0C00090F800044009082811D20121814011F094
:10D0D000EC0F0CD00C4882684FF480016AB10168F3
:10D0E00041F48001016010BD42F2010001E042F212
:10D0F0000200BDE81040FCF79FBB4FF0E020C0F8F5
:10D10000001110BD16E000E0AC4600207FB52A48B3
:10D1100000F15C01826B6846FFF7E8FA274E9DE854
:10D12000070006F11C03274C83E807001946244832
:10D13000C8600020A0706060A0604FF44771A6F541
:10D140004070FBF783F9A6F540721F4902F547705E
:10D15000FFF754F800282BD0A07858B3A6F54070FC
:10D1600090F86C11002901781CD019BB90F872015D
:10D1700000B3D4E90112A6F5C6756846FFF7B6FA02
:10D180009DE80F001C3686E80F004FF4B271284668
:10D19000FBF75CF92A460D493046FFF72FF80028C7
:10D1A00006D003E031B1807920B1094D0120E5605E
:10D1B00004B070BD0020FBE7383F0020B8450020D8
:10D1C0003DC502003823002070D6020050D5020071
:10D1D000C042002070B503466FF07F40814200D20C
:10D1E0000846124DD5F804250244081A411E22F0C3
:10D1F0007F425860952902D29630963A58601C7B3F
:10D2000005EB8400C0F8402509494FF4F8608847D1
:10D210004FF4A07000EB84012846FEF7F5FB4FF4B5
:10D220008030A040C5F8040370BD0000001001402C
:10D23000C1D4020070B5184E307800282AD11748A2
:10D2400000680125C0F3004008B915480560154C79
:10D250004FF480712046FEF7D7FB4FF4A0712046B3
:10D26000FEF7D2FB4FF4A2712046FEF7CDFB0E492C
:10D27000A02081F800044FF0E0224FF4003100209C
:10D28000C2F80011C4F80805A56025600220C4F8A2
:10D290000403357070BD0000D02200201804004047
:10D2A000080000400010014011E000E070B5154694
:10D2B0000E460446FFF7BEFF314620462560BDE816
:10D2C0007040FFF787BF0000017B4FF4803088403B
:10D2D0000149C1F808037047001001400870020AB4
:10D2E0004A70020C8A70000EC8700420704700005B
:10D2F00010B50248FDF73FFA002010BD582300206A
:10D3000010B514210448FBF7A1F804480068FDF7A4
:10D31000EBF9002010BD0000A448002024D8020032
:10D3200030B50F2490F8553000220BB1042B03D1F7
:10D3300090F86450012D06D0DD0707D090F85650C4
:10D34000012D02D002E0826E0DE0826D9B070AD5AE
:10D3500090F85C30012B06D1064B006EC3F53833D4
:10D36000984205D802440AB101240A60204630BD23
:10D370000424FBE70080020030B1006805498842C0
:10D3800005D048F20250704748F201507047002023
:10D39000704700006E52464870B5FEF7DFFC00286B
:10D3A00011D00020084A094B094C0121166801FAE6
:10D3B00000F52E4203D004EB8005C5F80036401C72
:10D3C000C0B20728F2D370BD080501403546526E41
:10D3D00000000140FFF7E0BF0020704700207047C9
:10D3E0002DE9FC4180461C4617460E460C48089D18
:10D3F000FDF7C4F910B11120BDE8FC81A20839463F
:10D400003046FEF7DFFA0648FDF7B5F933463A46EF
:10D4100001214046CDE90045FCF7EAFF0020EBE79B
:10D42000582300202DE9F84F114D884681461E46AD
:10D4300017466946DDF828A02868FDF770F9040052
:10D4400013D01C21FBF702F800202071C4F80090D3
:10D45000C4E90486C4E902A769462868FDF780F993
:10D46000FFF72EFB0020BDE8F88F0420FBE700004B
:10D4700024D80200CF3F998E73EBCA98FE897B5166
:10D48000A5E555658CE600777A1E7CD28DA4B8712F
:10D490000BAE51180822E3C7190C0E58A0DDE3BCEF
:10D4A000B5F7196FFEC0C1F88D347BB3F206FE9656
:10D4B0006C215E550D0E0F100B0C181900000000AA
:10D4C0000338FDD87047000051BD020057BD02006F
:10D4D0002DBD0200200000007800000000000000C8
:10D4E0004800280000204000A18702000000000042
:10D4F0000100010000000000010000000000000029
:10D5000002000500010000002200000000000000F1
:10D51000000000000000000000000000000000000B
:10D5200001000100000000000100000000000000F8
:10D5300002000500010000004200000000000000A1
:10D5400000000000000000000000000000000000DB
:10D55000010011000400FCFF0400000000000000B6
:10D56000020011000400FCFF0400000000000000A5
:10D57000030021000400FCFF040010000000000074
:10D58000040011000100FFFF010000000000000086
:10D59000050011000200FEFF040000000000000072
:10D5A000060011000400FCFF040000000000000061
:10D5B000070011000400FCFF040000000000000050
:10D5C000080017000200FEFF24000000F0D4020053
:10D5D000090010000100FFFF01000000ECD4020070
:10D5E0000A0027000200FEFF4400030020D50200CD
:10D5F000000000000000000000000000000000002B
:10D60000010011000100FFFF010000000000000008
:10D61000020017000200FEFF6401000050D5020066
:10D6200000000000000000000000000000000000FA
:10D6300001000700000000006801000000D60200A1
:10D6400002000100000000000100000000000000D6
:10D65000030005000100000042000000000000007F
:10D6600000000000000000000000000000000000BA
:10D67000010017000400FCFF6801000000D6020052
:10D68000020017000400FCFFAC01000030D60200CD
:10D69000000000000000000000000000000000008A
:10D6A000001103000011130002000000010000003F
:10D6B0000338FDD870470C000C0000005802000031
:10D6C0000200000000000000020000000000000056
:10D6D000A02700200900000000000000000000005A
:10D6E0000100000000000000280000000000000011
:10D6F0000000000000010000000001000000000028
:10D700000000000000000000000000000000000019
:10D71000D59A020000000000000000000000000098
:10D7200002000000000001000000000000000000F6
:10D730000800000000000000D59A020095BF02001A
:10D7400000000000000000000400000000000000D5
:10D7500000000000000000000000000000000000C9
:10D7600000000000000000000000000000000000B9
:10D77000F40000000000000018000000000000009D
:10D780000000000000000000000000000000000099
:10D790000000000000000000000000000000000089
:10D7A000170000000000000050EADA308883B89FBC
:10D7B000604F15F30000C98E020000000000000059
:10D7C0000000000000000000040000000000000055
:10D7D0000000000000000000000000000000000049
:10D7E0000001000000000000000000000000000038
:10D7F0000000000000000000001000000400000015
:10D8000001000000C5A50200F1D20200E5CA020035
:10D81000E1D302005DA30200B9CB0200D9D302001C
:10D8200009A60200B8460020001000000400000015
:10D8300001000000D1A5020001D30200F3CA0200DA
:10D8400025D40200A5A30200BDCB0200DDD3020057
:10D8500019A60200982F8A4291443771CFFBC0B5B8
:10D86000A5DBB5E95BC25639F111F159A4823F92AB
:10D87000D55E1CAB98AA07D8015B8312BE85312404
:10D88000C37D0C55745DBE72FEB1DE80A706DC9BC5
:10D8900074F19BC1C1699BE48647BEEFC69DC10F71
:10D8A000CCA10C246F2CE92DAA84744ADCA9B05CAD
:10D8B000DA88F97652513E986DC631A8C82703B070
:10D8C000C77F59BFF30BE0C64791A7D55163CA067E
:10D8D00067292914850AB72738211B2EFC6D2C4D8A
:10D8E000130D385354730A65BB0A6A762EC9C28178
:10D8F000852C7292A1E8BFA24B661AA8708B4BC20E
:10D90000A3516CC719E892D1240699D685350EF437
:10D9100070A06A1016C1A419086C371E4C774827EE
:10D92000B5BCB034B30C1C394AAAD84E4FCA9C5B64
:10D93000F36F2E68EE828F746F63A5781478C884B5
:10D940000802C78CFAFFBE90EB6C50A4F7A3F9BE97
:10D95000F27871C610DB020018DB02000000000044
:10D96000000000000200000754D9020064D9020040
:10D97000080000008CD902009CD9020008000000B9
:10D980009CD90200ACD902000800000030DB020084
:10D9900038DB0200000000000000000020DB020075
:10D9A00030DB02000000000000000000000000006A
:10D9B00000000000000000000000000008DB020082
:10D9C00010DB02000000000000000000C822002060
:10D9D000ACD90200CCD902000800000018DB02001C
:10D9E00020DB02000000000000000000DCD9020083
:10D9F000ECD9020008000000A5C102004DC10200E0
:10DA0000F5C002006BC0020071C0020029C0020014
:10DA100077C00200B5C0020000000000082000012D
:10DA2000FFFFFFFFFFFFFFFFFFFFFFFF0000000002
:10DA3000000000000000000001000000FFFFFFFFE9
:10DA4000512563FCC2CAB9F3849E17A7ADFAE6BCA0
:10DA5000FFFFFFFFFFFFFFFF00000000FFFFFFFFD2
:10DA600096C298D84539A1F4A033EB2D817D037778
:10DA7000F240A463E5E6BCF847422CE1F2D1176B13
:10DA8000F551BF376840B6CBCE5E316B5733CE2BE6
:10DA9000169E0F7C4AEBE78E9B7F1AFEE242E34F15
:10DAA0004B60D2273E3CCE3BF6B053CCB0061D6552
:10DAB000BC86987655BDEBB3E7933AAAD835C65ADB
:10DAC0004F860200E99302000592020044DB020047
:10DAD000C8220020B8000000E4960200FCDB02002F
:10DAE00080230020382D0000F4960200ED9B0200F8
:10DAF0008D9B020018230020F02700200128002021
:10DB000004280020F4000000859C020000000000B2
:10DB100015B80200000000004DB80200000000002F
:10DB2000D1BA02000000000045BC02000000000065
:10DB30002DB80200000000000000000003000000FB
:10DB400041B10200000000000000000000000000E1
:10DB5000E0220020F0220020000000000000000071
:10DB600000000000000000000000000000000000B5
:10DB700000000000000000000100000000000000A4
:10DB800000000000FF00FFFF000000000000000098
:10DB90000000000000000000000000000000000085
:10DBA0000100000000000000000000000000000074
:10DBB00000E0020000000000000000000000000083
:10DBC0000000000000000000000000000000000055
:10DBD0000000000000000000000000000000000045
:10DBE000000000000090D0030000000000000000D2
:0CDBF0007DA202000010000000000300F5
:020000041000EA
:041014000080020056
:020000041000EA
:0410180000E00200F2
:040000050002820172
:00000001FF
